:100000000C9435000C945D000C945D000C945D0024
:100010000C945D000C945D000C945D000C945D00EC
:100020000C945D000C945D000C945D000C945D00DC
:100030000C945D000C945D000C945D000C945D00CC
:100040000C9491010C945D000C9401020C94DB0162
:100050000C945D000C945D000C945D000C945D00AC
:100060000C945D000C945D00EB0211241FBECFEFD9
:10007000D8E0DEBFCDBF11E0A0E0B1E0E0E4F6E003
:1000800002C005900D92AE39B107D9F722E0AEE972
:10009000B1E001C01D92A434B207E1F710E0C5E35E
:1000A000D0E004C02197FE010E941803C433D10799
:1000B000C9F70E9433020C941E030C9400003FB752
:1000C000F8948091400290914102A0914202B09137
:1000D000430226B5A89B05C02F3F19F00196A11D2C
:1000E000B11D3FBFBA2FA92F982F8827BC01CD0182
:1000F000620F711D811D911D42E0660F771F881FE1
:10010000991F4A95D1F70895AF92BF92CF92DF928F
:10011000EF92FF920F931F93CF93DF936C017B01BC
:100120008B01040F151FEB015E01AE18BF08C0174D
:10013000D10759F06991D601ED91FC910190F081C0
:10014000E02DC6010995892B79F7C501DF91CF9183
:100150001F910F91FF90EF90DF90CF90BF90AF90E5
:100160000895FC01538D448D252F30E0842F90E0BD
:10017000821B930B541710F0CF96089501970895A2
:10018000FC01918D828D981761F0A28DAE0FBF2F6B
:10019000B11D5D968C91928D9F5F9F73928F90E0C1
:1001A00008958FEF9FEF0895FC01918D828D981730
:1001B00031F0828DE80FF11D858D90E008958FEF6D
:1001C0009FEF0895FC01918D228D892F90E0805C36
:1001D0009F4F821B91098F73992708958EE991E0B3
:1001E0000E94E20021E0892B09F420E0822F08958B
:1001F00080E090E0892B29F00E94EE0081110C94A0
:1002000000000895FC01A48DA80FB92FB11DA35AB9
:10021000BF4F2C91848D90E001968F739927848F26
:10022000A689B7892C93A089B1898C918370806449
:100230008C93938D848D981306C00288F389E02DEA
:1002400080818F7D80830895EF92FF920F931F939B
:10025000CF93DF93EC0181E0888F9B8D8C8D981379
:100260001AC0E889F989808185FF15C09FB7F89485
:10027000EE89FF896083E889F989808183708064D1
:1002800080839FBF81E090E0DF91CF911F910F911C
:10029000FF90EF900895F62E0B8D10E00F5F1F4F2B
:1002A0000F731127E02E8C8D8E110CC00FB607FC3A
:1002B000FACFE889F989808185FFF5CFCE010E94C8
:1002C0000201F1CFEB8DEC0FFD2FF11DE35AFF4F33
:1002D000F0829FB7F8940B8FEA89FB898081806256
:1002E000CFCFCF93DF93EC01888D8823B9F0AA8913
:1002F000BB89E889F9898C9185FD03C0808186FDE1
:100300000DC00FB607FCF7CF8C9185FFF2CF80812F
:1003100085FFEDCFCE010E940201E9CFDF91CF91A1
:1003200008951F920F920FB60F9211242F933F93AF
:100330008F939F93AF93BF9380913C0290913D0226
:10034000A0913E02B0913F0230913B0223E0230F87
:100350002D3758F50196A11DB11D20933B028093C6
:100360003C0290933D02A0933E02B0933F028091E5
:10037000400290914102A0914202B0914302019645
:10038000A11DB11D8093400290934102A0934202AF
:10039000B0934302BF91AF919F918F913F912F9165
:1003A0000F900FBE0F901F90189526E8230F02960E
:1003B000A11DB11DD2CF1F920F920FB60F92112423
:1003C0002F933F934F935F936F937F938F939F935D
:1003D000AF93BF93EF93FF938EE991E00E940201E8
:1003E000FF91EF91BF91AF919F918F917F916F910D
:1003F0005F914F913F912F910F900FBE0F901F90E3
:1004000018951F920F920FB60F9211242F938F936E
:100410009F93EF93FF93E091AE01F091AF01808144
:10042000E091B401F091B50182FD1BC090818091F3
:10043000B7018F5F8F732091B801821741F0E0916F
:10044000B701F0E0E256FE4F958F8093B701FF9120
:10045000EF919F918F912F910F900FBE0F901F9052
:1004600018958081F4CF789484B5826084BD84B57A
:10047000816084BD85B5826085BD85B5816085BD9F
:1004800080916E00816080936E0010928100809157
:1004900081008260809381008091810081608093DF
:1004A0008100809180008160809380008091B10004
:1004B00084608093B1008091B00081608093B0002F
:1004C00080917A00846080937A0080917A008260C3
:1004D00080937A0080917A00816080937A00809185
:1004E0007A00806880937A001092C100E091AE019A
:1004F000F091AF0182E08083E091AA01F091AB011D
:100500001082E091AC01F091AD018FEC80831092EC
:10051000B601E091B201F091B30186E08083E091F1
:10052000B001F091B101808180618083E091B001E0
:10053000F091B101808188608083E091B001F091F9
:10054000B101808180688083E091B001F091B101B8
:1005500080818F7D8083C0E0D0E048E850E062E198
:1005600071E08EE991E00E94840042E050E06BE986
:1005700071E08EE991E00E9484000E945F004B01CF
:100580005C0188EBC82E8BE0D82EE12CF12C0E9468
:100590005F00681979098A099B09683E73408105E3
:1005A0009105A8F321E0C21AD108E108F10888EE0C
:1005B000880E83E0981EA11CB11CC114D104E10473
:1005C000F10429F7209749F20E94EE00882329F2CE
:1005D0000E940000C2CFEEE9F1E01382128288EEA1
:1005E00093E0A0E0B0E084839583A683B78384E0A2
:1005F00091E09183808385EC90E09587848784ECFB
:1006000090E09787868780EC90E0918B808B81ECDF
:1006100090E0938B828B82EC90E0958B848B86ECC0
:1006200090E0978B868B118E128E138E148E089508
:10063000EE0FFF1F0590F491E02D0994F894FFCF81
:100640000000000024018400B1007101E200C0003C
:10065000D400513239755A334A6864485673595830
:100660005270623234734948526F5A53426D624736
:10067000466E49475A766369416E546D39316379E4
:100680004268646D39756379446749475A686158AF
:100690004A6C494F416764573467633256796157F2
:1006A0004673494774706247786C63696367615841
:1006B0004D674F69424456455974524578546530E8
:1006C000517A6331396E4D32356A6158597A6331E6
:0E06D000387958334177636D4E39000D0A00BA
:00000001FF
